:10275200000100030018000602050505060606062C
:10276200070707080809090A0B0C0C0D0E101213B3
:1027720015171B1E252A2F363A3B37312C26231ECE
:0B2782001D18181515131111100F0F72
:101F9600C10B019B01019100019A00C10AC1000118
:101FA6001300010800011B004200F1012C4100AAA8
:101FB600004100CF00011A00C103C182C108C1015E
:071FC6004100F314010D00BE
:10191C0012176E9000FFE0540C640C6029D2043056
:10192C00091FC209E51DD394004009D51D061229D3
:10193C00A012297A7854E6600816E6B4010312283E
:10194C00EA1229BA80CD12287C300934C209789A5F
:10195C0006E51DD394004009D51D061229A01229B5
:10196C007A7854E6600B16E6B401062005031228BB
:10197C00EA789AE6D3940A4007E4F6C20C120EAF4A
:10198C007888E6D39427403AE4F61229BA12246FE9
:10199C00E4F519E51925E02493F9E7FF789CF66046
:1019AC001816E6FFFDE51925E02492F8760008A646
:1019BC0005EF7005AF1912294A0519E519C39404EE
:1019CC0040D17891E6608216E62410F8E614601394
:1019DC0024FE6016240370EA12028CE4FDFF122729
:1019EC008D80DFB204121BF480D8200A03021A8CFB
:1019FC00C39000BBE09402503CC207A20630070122
:101A0C00B35021C2069000FFE0547FF0FD7C007FB4
:101A1C00631206FB9000EEE04480F0A3E0F090002F
:101A2C00F37414F0E4F527F5287B89FA7D147F1400
:101A3C0012136C804BD39000BCE094009000BBE080
:101A4C009402403CD207A206300701B35021D206C3
:101A5C009000FFE04480F0FD7C007F631206FB9059
:101A6C0000EEE04480F0A3E0F09000F37414F07505
:101A7C0027007528047B897A007D147F1412136C5F
:0A1A8C00E4FD7F0312278D0219CE3E
:10176E00300012D2A0D2A1D2A2D2A3D2A4D2A5D29C
:10177E00A6D2A78010C2A0C2A1C2A2C2A3C2A4C2F6
:10178E00A5C2A6C2A7D2B4D294D295C2B7C2B5C2D0
:10179E00B6C2D9C2B37580FF759850758921758709
:1017AE0080758DFD758BFD758A04758CF7D28ED282
:1017BE008CD2A943BF021228367D037C007F04120F
:1017CE0006FBD2AFD2AC750B011229BA7F507EC385
:1017DE0012297E1229BA7F507EC312297E1229BA8F
:1017EE007F507EC312297E1229BA7F507EC31229E2
:1017FE007E1229BA7F507EC312297E1229BAE4F5D1
:10180E000BF523E52325E024ABF582E43400F583C4
:10181E00E4F0A3F00523E523B412E87B007A007907
:10182E00247F041226D7EF602BE524640360487DE5
:10183E00037C007F041206FBE4FDFC7F631206FBB3
:10184E007D807C007F0A1206FB7D017C007F0912E1
:10185E0006FB80237D037C007F041206FBE4FDFC67
:10186E007F631206FB7D807C007F0A1206FB7D01E2
:10187E007C007F091206FB7B017A0079FF7F6312E1
:10188E0026D7EF70049000FFF07B017A0079F07F8D
:10189E000A1226D7EF700E9000F07480F0FD7C00D7
:1018AE007F0A1206FB7B017A0079F67F091226D792
:1018BE00EF700D9000F604F0FD7C007F091206FB20
:1018CE007B007A0079087F081226D7E4FD7F01128B
:1018DE00278DE4FDFF12278D9000F6E06402702D37
:1018EE00FD7F0312278DE4F523E52325E024D0F5B3
:1018FE0082E43400F583E4F0A3F00523E523B4106D
:0D190E00E89000FFE030E703D20622C20699
:01191B0022A9
:03000B000225F2D9
:1025F200C0E0C0F0C083C082C0D075D000C000C0AF
:1026020001C002C003C004C005C006C007758A0429
:10261200758CF7788806D209789B06E6D394034036
:102622000276011222ECD007D006D005D004D003E6
:10263200D002D001D000D0D0D082D083D0F0D0E070
:012642003265
:10294A007891E6C394035007E6062410F8A60722F6
:10278D00ED701FEF25E02452F582E43427F583E444
:10279D0093FA740193FBEF25E02492F8A60208A6A4
:0F27AD000322EDEF25E02492F8760008A605221E
:10287C00E5087006439B4075A303E508C39401402B
:0D288C0002D20AE508C394034002D20022E4
:081A96008B3A8A3B893C8D3D2F
:101A9E00E4F53FE53FC3953D4003021BF3AB3AAA85
:101AAE003BA93CE53F0475F002A4F58285F0831254
:101ABE000E20FFAEF0E53F253E25E024ABF582E497
:101ACE003400F583E0FCA3E0FDC3EF9DFDEE9CFC2E
:101ADE00C3ED9414EC64809480500BC3ED94ECEC45
:101AEE006480947F5014E53F253E25E024ABF582BB
:101AFE00E43400F583EEF0A3EFF0AB3AAA3BA93C39
:101B0E00E53F0475F002A4F58285F083120E20FFE6
:101B1E00E53F253EFD25E024ABF582E43400F58358
:101B2E00E0FAA3E0C39FEA95F0500D74F72DF5820D
:101B3E00E43400F583E004F0AB3AAA3BA93CE53F60
:101B4E000475F002A4F58285F083120E20FFE53FA6
:101B5E00253EF925E024ABF582E43400F583E0FC64
:101B6E00A3E0D39FEC95F0400D74F729F582E43491
:101B7E0000F583E014F074F729F582E43400F58360
:101B8E00E0D36480948A4023E53F253EFF25E02480
:101B9E00ABF582E43400F583E475F001120DDF74C9
:101BAE00F72FF582E43400F583E4F074F729F5821B
:101BBE00E43400F583E0C3648094765023E53F253A
:101BCE003EFF25E024ABF582E43400F58374FFF587
:101BDE00F0120DDF74F72FF582E43400F583E4F094
:051BEE00053F021AA1F1
:011BF30022CF
:101BF400200A02D2B2C293D20C7F08121EC1D29321
:101C0400200803021CED300A67E4F523E52325E0F0
:101C140024ABF582E43400F583E0FEA3E0FFD39423
:101C240064EE94005019E52325E024BBF582E434E6
:101C340000F583E0FCA3E0D39464EC94004022C359
:101C4400EF9484EE9403401FE52325E024BBF58242
:101C5400E43400F583E0FEA3E0C39484EE940340EF
:101C6400069000CFE004F00523E523B4089E8068C5
:101C7400E4F523E52325E024BBF582E43400F58371
:101C8400E0FEA3E0FFE52325E024ABF582E4340085
:101C9400F583E0FCA3E0C39FFFEC9EFE122927D34B
:101CA400EF9432EE6480948040259000CFE004F0FD
:101CB40074079523FFE51AA807088003A2E713D841
:101CC400FB4401FEA807088002C333D8FCF51A05BB
:101CD40023E523C39408409B9000CFE0B4FF06C2E1
:101CE40002C2088004D202C208E4FD7F0102278DEB
:100EAF00E4F526858025A2B7920DA2B5920EA2B6C3
:100EBF00920FC2B7C2B5C2B67580FF200C04C2B480
:100ECF008002C21112297A200C09C294858023D284
:100EDF00948007C213858023D2137580FF200C09DD
:100EEF00C295858024D2958007C212858024D212A4
:100EFF00D2B47D01E4FCE5235D7003D38001C350C0
:100F0F000AE5245D70028001C34003ED4226ED2502
:100F1F00E0FD0CBC08E0852580A20D92B7A20E92D1
:100F2F00B5A20F92B6A20CE433FF2418F8E665269B
:100F3F006027A20CE433FE240FF806740F2EF8E698
:100F4F00C3940A401AA20CE433FE2418F8A62674A0
:100F5F000F2EF8E4F6D2108006740F2FF8E4F6A2E5
:100F6F000CE433FF240CF8E665236027A20CE4336E
:100F7F00FE240AF806740A2EF8E6C3940A401AA251
:100F8F000CE433FE240CF8A623740A2EF8E4F6D2F0
:100F9F00108006740A2FF8E4F6A20CE433FF24172E
:100FAF00F8E665246027A20CE433FE240EF80674DD
:100FBF000E2EF8E6C3940A401AA20CE433FE24174F
:100FCF00F8A624740E2EF8E4F6D2108006740E2FB5
:100FDF00F8E4F67D012010030210E2C210200C7A13
:100FEF00E4FCA20CE433FF2418F8E65D7008748962
:100FFF002CF8E4F68026740C2FF8E65D70087489DF
:10100F002CF87601801674172FF8E65D7008748936
:10101F002CF87602800674892CF8E4F6ED25E0FDB5
:10102F000CBC08BEE49000CBF0A3F0FC9000CBE02A
:10103F00FEA3E07802C333CE33CED8F9FF9000CBB6
:10104F00EEF0A3EFF074892CF8E6FBEE9000CBF0F6
:10105F00EB4FA3F00CBC08D480797C08A20CE433CE
:10106F00FF2418F8E65D700874892CF8E4F68026E2
:10107F00740C2FF8E65D700874892CF876018016D1
:10108F0074172FF8E65D700874892CF876028006C5
:10109F0074892CF8E4F6ED25E0FD0CBC10BEE4904D
:1010AF0000CDF0A3F07C089000CDE0FEA3E0780225
:1010BF00C333CE33CED8F9FF9000CDEEF0A3EFF0CF
:1010CF0074892CF8E6FBEE9000CDF0EB4FA3F00CFB
:1010DF00BC10D4200C4B9000F6E0FF70219000CB99
:1010EF00E0FCA3E0FD4C6010ED64AA7003EC64AA71
:1010FF006006BC5506BD5503D20322C20322EF7012
:10110F00209000CDE0FEA3E0FF4E6010EF64AA70C8
:10111F0003EE64AA6006BE5506BF5503D20322C272
:01112F0003BC
:01113000229C
:10028C00E4F525F526200A1ED2939000F5E0FF1325
:10029C009290EFA2E19291A2E29292C2B27FF47E8E
:1002AC000112297ED2B29000F5E0045407F0A3E0CD
:1002BC00F960030203C8300A6E2002030203C890DF
:1002CC0000AAE0640C7057E513045407F513C2023E
:1002DC00D20830012625E024ABF582E43400F58306
:1002EC007403F0A374E8F0E513B40702C201E490C0
:1002FC0000AAF0E50B6027150B8023E51325E024FD
:10030C00ABF582E43400F583E4F0A3F0E513B40715
:10031C0002D201E49000AAF0E50B6002150B9000EC
:10032C00AAE004F00203C82002030203C89000F5FF
:10033C00E0FF30E0159000F1E0FCA3E0FDC374E8B1
:10034C009DF52474039CF523800A9000F1E0F523BD
:10035C00A3E0F524C374079F25E024ABF582E434B5
:10036C0000F583E523F0A3E524F09000AAE06420D7
:10037C007044C202D20830011B9000F2E02464F0F9
:10038C009000F1E03400F0E0B40320A3E0B4E81BEB
:10039C00C20180179000F2E0249CF09000F1E03450
:1003AC00FFF0E07002A3E07002D201E49000AAF02A
:1003BC00E50B6002150B9000AAE004F0200A030282
:1003CC0006919000F5E0FFB4080040030206FA9095
:1003DC0003E2F82828730203FA0204480204990283
:1003EC0004ED0205410205950205E902063D7489FA
:1003FC002FF8E6FE700CE96009300003C2A022D28F
:10040C00A022EEB4010CE96009300003D2A022C294
:10041C00A022EF25E024ABF582E43400F583E0FC68
:10042C00A3E0C394E8EC94034009300003D2A0226B
:10043C00C2A022300003C2A022D2A02274892FF8BD
:10044C00E6FF700CE96009300003C2A122D2A122A0
:10045C00EFB4010CE96009300003D2A122C2A12241
:10046C009000F5E025E024ABF582E43400F583E060
:10047C00FEA3E0C394E8EE94034009300003D2A13C
:10048C0022C2A122300003C2A122D2A1229000F5E7
:10049C00E02489F8E6FF700CE96009300003C2A281
:1004AC0022D2A222EFB4010CE96009300003D2A2DF
:1004BC0022C2A2229000F5E025E024ABF582E434C0
:1004CC0000F583E0FEA3E0C394E8EE94034009300A
:1004DC000003D2A222C2A222300003C2A222D2A2C4
:1004EC00229000F5E02489F8E6FF700CE9600930F1
:1004FC000003C2A322D2A322EFB4010CE96009309D
:10050C000003D2A322C2A3229000F5E025E024AB85
:10051C00F582E43400F583E0FEA3E0C394E8EE94A6
:10052C00034009300003D2A322C2A322300003C22D
:10053C00A322D2A3229000F5E02489F8E6FF700CE8
:10054C00E96009300003C2A422D2A422EFB4010C4A
:10055C00E96009300003D2A422C2A4229000F5E085
:10056C0025E024ABF582E43400F583E0FEA3E0C380
:10057C0094E8EE94034009300003D2A422C2A422D2
:10058C00300003C2A422D2A4229000F5E02489F802
:10059C00E6FF700CE96009300003C2A522D2A52247
:1005AC00EFB4010CE96009300003D2A522C2A522E8
:1005BC009000F5E025E024ABF582E43400F583E00F
:1005CC00FEA3E0C394E8EE94034009300003D2A5E7
:1005DC0022C2A522300003C2A522D2A5229000F58A
:1005EC00E02489F8E6FF700CE96009300003C2A62C
:1005FC0022D2A622EFB4010CE96009300003D2A686
:10060C0022C2A6229000F5E025E024ABF582E4346A
:10061C0000F583E0FEA3E0C394E8EE9403400930B8
:10062C000003D2A622C2A622300003C2A622D2A662
:10063C00229000F5E02489F8E6FF700CE96009309F
:10064C000003C2A722D2A722EFB4010CE960093043
:10065C000003D2A722C2A7229000F5E025E024AB2C
:10066C00F582E43400F583E0FEA3E0C394E8EE9455
:10067C00034009300003D2A722C2A722300003C2D4
:10068C00A722D2A7229000F5E02489F8E6FF700893
:10069C00A3E06004E4F5A722EFB401179000F6E0A4
:1006AC0060119000F0E02468FFE43403FE1221BADC
:1006BC008FA7229000F5E0FFC374079F25E024ABC1
:1006CC00F582E43400F583E0FEA3E0FF9000F0E057
:1006DC00FD7C00EF2DFFEC3ECF2480CF34FFFEC31A
:0E06EC00648094805003E4FEFF1221BA8FA7B1
:0106FA0022DD
:10246F00E4FF74892FF8E6FEB4021FEF25E024ABDA
:10247F00F582E43400F583E0FCA3E0D394F4EC940C
:10248F00014007E51413F5148014EEB40108E514A8
:10249F00C313F5148008E514C3134480F5140FBF5C
:1024AF0008C0E4FFEF25E024BBF582E43400F58398
:1024BF00E0FCA3E0D39400EC94024007E51613F57B
:0F24CF00168008E516C3134480F5160FBF08D515
:0124DE0022DB
:1022EC007580FF789BE624FE601A146067240270E8
:1022FC0078C2B5C2B6E50B6005E4F58080038514A1
:10230C0080D2B722C2B7C2B612297A9000F6E0701A
:10231C00183004055315FE80034315013003055393
:10232C0015FD8021431502801C3004055315FE80D9
:10233C0003431501E509D39400400715095315FD16
:10234C008003431502E50B6005E4F58080038515D9
:10235C0080D2B522C2B7C2B512297AE50B6005E46A
:0A236C00F5808003851680D2B622AA
:0429BA00759FA7223C
:04297A007F0A7E0052
:0B297E00EF1FAC0670011E4C70F6222B
:0421BA008E278F28B5
:1021BE00E4F52990275A93752A00F52BD3E52B9534
:1021CE0028E52A95274006E4FAFBFFFE220529AFF3
:1021DE0029EF3395E0FE745A2FF58274273EF5836E
:1021EE00E493F9252BF52BE4352AF52AD3E52B9527
:1021FE0028E52A95274050E52B9528FFE52A9527B7
:10220E00FEE9C39FFBE49EFA7C007D0AAF03FE123B
:10221E000D42AA06AB07E9FD120DA9AA06AB077C73
:10222E00007D05120D427D0A120DA9AA06AB07AF5D
:10223E0029EF3395E0FE7C007D05120D42EF2BFB5E
:10224E00EE3AFAAF03FE22E5297082FA7BFF7FFF9A
:01225E00FE81
:01225F00225C
:10156E0000C1814001C0804101C0804100C1814065
:10157E0001C0804100C1814000C1814001C0804155
:10158E0001C0804100C1814000C1814001C0804145
:10159E0000C1814001C0804101C0804100C1814035
:1015AE0001C0804100C1814000C1814001C0804125
:1015BE0000C1814001C0804101C0804100C1814015
:1015CE0000C1814001C0804101C0804100C1814005
:1015DE0001C0804100C1814000C1814001C08041F5
:1015EE0001C0804100C1814000C1814001C08041E5
:1015FE0000C1814001C0804101C0804100C18140D5
:10160E0000C1814001C0804101C0804100C18140C4
:10161E0001C0804100C1814000C1814001C08041B4
:10162E0000C1814001C0804101C0804100C18140A4
:10163E0001C0804100C1814000C1814001C0804194
:10164E0001C0804100C1814000C1814001C0804184
:10165E0000C1814001C0804101C0804100C1814074
:10166E0000C0C101C30302C2C60607C705C5C40434
:10167E00CC0C0DCD0FCFCE0E0ACACB0BC90908C8A4
:10168E00D81819D91BDBDA1A1EDEDF1FDD1D1CDC94
:10169E0014D4D515D71716D6D21213D311D1D01004
:1016AE00F03031F133F3F23236F6F737F53534F4F4
:1016BE003CFCFD3DFF3F3EFEFA3A3BFB39F9F83864
:1016CE0028E8E929EB2B2AEAEE2E2FEF2DEDEC2C54
:1016DE00E42425E527E7E62622E2E323E12120E0C4
:1016EE00A06061A163A3A26266A6A767A56564A4B4
:1016FE006CACAD6DAF6F6EAEAA6A6BAB69A9A86824
:10170E0078B8B979BB7B7ABABE7E7FBF7DBDBC7C13
:10171E00B47475B577B7B67672B2B373B17170B083
:10172E005090915193535292965657975595945473
:10173E009C5C5D9D5F9F9E5E5A9A9B5B99595898E3
:10174E00884849894B8B8A4A4E8E8F4F8D4D4C8CD3
:10175E004484854587474686824243834181804043
:051FCD00015200C114E7
:10283600C2D8E47852F67854F6FB7A00791E7F0601
:102846001226D7EF7003751EFEE51E6003B4FF0364
:04285600751EFE22CB
:0A29A000C2D8E47852F67854F6220B
:0B299500C215D2D87F0A7E0002297E06
:030023000223F7BE
:1023F700C0E0C0D075D000C000C006C007309856F6
:102407007852E6C394325007E6062456F8A699C2D6
:10241700987852E6FFB40105751D328040EF6406D7
:1024270070257857E6FE64036004EEB40605751C54
:1024370008802AEEB4100B785BE625E02409F51C2A
:10244700801B751C328016EFB51C12751D00785461
:102457007606D2168007309904C299D215D007D0D4
:0824670006D000D0D0D0E03215
:1028EA00122058500F7509141229951229AA120993
:0728FA00901211310229A028
:102058007858E6FE08E6F97C002400FFEC3EFE789E
:1020680052E6651C6002C3227856E6FDF4600AED6C
:10207800651E6005ED6002C3227857E6FD640360C3
:102088000CED64066007ED64106002C322ED64067F
:102098007041C3EF9408EE94005038E9C39402509D
:1020A800099000FFE030E02BC322E9C394045009F3
:1020B8009000FFE030E11CC322E9B408099000FF5A
:1020C800E030E20FC322E9B407099000FFE030E3F3
:1020D80002C3227B007A007956E51C24FEFD1226F5
:1020E80094AD07AC067454251CF8E6FE7455251CFF
:1020F800F8E67A002400FFEA3EFEEFB50506EEB5E5
:052108000402D322C314
:01210D0022AF
:10113100E4F5287857E6B4061FE4F5287456252807
:10114100F8E6F5997F327E0012297E1229BA052828
:10115100E528C3940840E5227857E664036003025A
:10116100132E08E6FE08E67C002400F524EC3EF58B
:1011710023785BE6F5277856E6F529F59912289C40
:101181007857E6F5293015FD122899E52725E0F570
:10119100293015FD122899C3E5249464E5239400B0
:1011A1004003021241E528C395274003021241E59D
:1011B10028C3946440030212417E00E5242528FFE0
:1011C100EE3523FEEF64634E7016F5293015FD12DE
:1011D10028999000FFE0F5293015FD122899805BD0
:1011E100E5282524FF7B007A007925122643EF703C
:1011F10004F525F5267E00E5242528FFEE3523FE9E
:10120100C3EF945AEE94004005E4F5298004E525E6
:10121100F5293015FD1228997E00E5242528FFEED9
:101221003523FEC3EF945AEE94004005E4F529807E
:1012310004E526F5293015FD12289905280211A685
:10124100E528C3952740030213157E00E5242528D0
:10125100FFEE3523FEC3EF9464EE940050030213B6
:1012610015E528C3952740030213157E00E52425C3
:1012710028FFEE3523FEEF64844E7017F5293015F3
:10128100FD1228999000FFE0F5293015FD122899EB
:10129100021310AF287E00E5242528CFEE3523CF99
:1012A100249CCF34FFFEC3EF9412EE9400504E7E87
:1012B10000E5242528FFEE3523FEEF25E0FFEE3380
:1012C100FE74E32FF58274FF3EF583E0F5293015B6
:1012D100FD1228997E00E5242528FFEE3523FEEF37
:1012E10025E0FFEE33FE74E32FF58274FF3EF583B4
:1012F100E0A3E0F5293015FD1228998012E4F529C3
:101301003015FD1228997529013015FD122899050E
:10131100280212623015FD7851E6F599C215301593
:10132100FD7853E6F599C21520153F80FB7857E605
:1013310064107036F52874562528F8E6F529F599D4
:10134100C2153015FDAF291228A01229BA0528E5CA
:1013510028C3940640E07851E6F599C2153015FD91
:0A1361007853E6F599C2153015FD2A
:01136B00225F
:10099000752C01C20C7857E664066003020B7408DC
:1009A000E6FE08E6FD7A002400FFEA3EFEC3EF946F
:1009B00064EE94004003020AECED9401502408E632
:1009C000FE08E67C002400FDEC3EFCE4FF1206FB82
:1009D0009000FFE04401F0FD7C007F631206FB0203
:1009E0000BC17859E6D39403502408E6FE08E67C50
:1009F000002400FDEC3EFC7F021206FB9000FFE0AD
:100A00004402F0FD7C007F631206FB020BC17859A3
:100A1000E66408702908E6FE08E67C002400FDEC88
:100A20003EFC7F081206FB9000FFE04404F0FD7CD2
:100A3000007F631206FB785BE6F508020BC178596C
:100A4000E66407702908E6FE08E67C002400FDEC59
:100A50003EFC7F071206FB9000FFE04408F0FD7C9F
:100A6000007F631206FB785BE6F51B020BC1785929
:100A7000E6FFB40613785BE6FD7C001206FB785BAC
:100A8000E6F51ED20C020BC17859E6FFB40A1378C2
:100A90005BE6FD7C001206FB785BE69000F0F0025E
:100AA0000BC17859E6FFB4091B785BE6FD7C0012A8
:100AB00006FB785BE69000F6F06003020BC1750B55
:100AC00001020BC17859E6FFB41011785BE6FD7C9A
:100AD000001206FB785BE6F52C020BC17859E6FFA5
:100AE000785BE6FD7C001206FB020BC17858E67FBE
:100AF00000FE08E67C002400FFEC3ECF249CF52895
:100B0000EF34FFF527D3E5289412E52794005043EE
:100B100008E6FE08E62400F524EC3EF523D3E524A0
:100B200094FFE523648094834003020BC17858E668
:100B3000FE08E62400FFEC3EFEEF25E0FFEE33FE6C
:100B400074E32FF58274FF3EF583E523F0A3E524DB
:100B5000F0806EE528646345277066785BE6752350
:100B600000F524FDAC237F631206FB785BE6900062
:100B7000FFF0804D7857E664107046785BE6F52B01
:100B80007858E6FE08E67C002400F528EC3EF527C0
:100B9000E4F529F52AC3E52A952BE529940050218F
:100BA0001229BAAF2AEF25E0245EF8E6FD7C00EFBB
:100BB000785926FF1206FB052AE52A70D8052980F8
:100BC000D4E52C647F7036752D77AF2D1228D2E4D2
:100BD000F5257B007A007926AF251226D7EF600D28
:100BE000E42525FDE434EEFCAF261228600525E55A
:100BF00025D3941040DCC2AF759F8080FE300C146A
:100C00001229BA752D77AF2D1228D27D067CEEAF52
:100C10001E122860E52CB4FF07C2AF759F8080FECE
:010C200022B1
:0929AA00785376FF785176FF2284
:07289900852999C215AF2942
:1028A0007851E66FFF90156E937853667951F7EF84
:0528B00090166E93F686
:0128B5002200
:082694008B238A2489258D2681
:10269C007527007528FF7DFFAF261526EF6026AB4A
:1026AC00230525E525AA247002052414F9120D171B
:1026BC006528FF90156E936D752700F528EF901621
:0A26CC006E93FD80D3E528FEEDFFBC
:0126D60022E1
:022901000000D4
:021EC1008F246C
:101EC30078257C007D007BFF7A2979017E007F14D1
:101ED300120CF1C290C291C292122915300C077FE5
:101EE300B11228108008200C057FB21228107F0140
:101EF3007E0012297E1227E7EF4E60030229B37F8B
:101F0300017E0012297E1227168E258F2675390130
:101F13001227BC7F017E0012297EE539139290E5DA
:101F230039A2E19291A2E29292122716E53925E0B5
:101F33002425F8A60608A6070539E539D3940940F0
:101F4300CF1229B3E5262528CFE5253527CF252A26
:101F5300CF3529CF252CCF352BCF252ECF352DCFE0
:101F63002530CF352FCF2532CF3531CF2534CF355F
:101F730033CF2536CF35355403FEE538B50713E5A2
:101F830037B5060E7B007A00792585243E7D08123D
:021F93001A969C
:011F95002229
:10291500C2DB7F057E0012297EC2DA7F027E0002BD
:02292500297E09
:1027BC00E4FFFE20DB0C0FBF00010EEF64644E70D3
:1027CC00F222D2DB7F017E0012297ED2DAC2DB7FBD
:0A27DC00017E0012297ED2DBC2DA72
:0127E60022D0
:022810008F3AFD
:10281200753B087F017E0012297EE53A3392DBD2B6
:10282200DA7F017E0012297EC2DAE53A25E0F53A26
:03283200D53BE0B3
:012835002280
:10271600E4F53BF53CF53AD2DA7F017E0012297EDC
:10272600E53C25E0FFE53B33FEA2DBE433FDEEF5B9
:102736003BEF4DF53CC2DA7F017E0012297E053A59
:0B274600E53AC3940A40D0AE3BAF3C24
:012751002265
:0729B300C2DBD2DAD2DB2205
:1027E700E4FDFCD2DBD2DAFBFAA2DBE4337C00FDAA
:1027F7007005C2DAFEFF220BBB00010AEB640A4A2E
:0828070070E7C2DA7E007F01D8
:01280F0022A6
:0B2989008F828E83E493120D307F01DB
:012994002220
:06285A00FEAD07FC7F3318
:10286000AB0775F65575F6AA75F65543BF048CF49B
:0C287000AF058FF58BF675F7807F002216
:1028D20075F65575F6AA75F65543BF04EF25E0F572
:0828E200F4E4F5F575F782221C
:0625A0008B4E8A4F8950AA
:1025A600120DF5FBAAF0530201EB24FFFFEA34FFFC
:1025B600FE7C007D0F120D54A905EB241DFFE43AA5
:1025C600FEE97C00C3EF9DFFEE9CFED3EF94FFEE89
:1025D600940140037F0022C3740F9DFFE49CAB4E21
:0B25E600AA4FA9508FF0120E587F0181
:0125F10022C7
:082546008F458B468A47894846
:10254E001229BAE54525E0F549754A00854A82F516
:10255E0083E493B433037F0022054AE54A700205F3
:10256E0049854A82854983E493B4FF14AB46AA4752
:10257E00A948E549854AF0120E901229BA7F012228
:10258E007B007A0079491225A0EF70D51229BA7F07
:01259E00003C
:01259F002219
:0E28B600AF3D1229398F42FB7A007932AF2EE6
:0E28C400EF75F0148425E025422463020D30E8
:02295A00AC07C8
:0E295C00ED25E07B00FAAF04FC7D0002286050
:06296A00AD34AC33E4FFC4
:0A297000ED2401FDE43CFC022860A8
:10293900AE07BE01037F0222BE02037F01227F0090
:01294900226B
:082376007A007933AD31AF2E7E
:0A237E008F458D468B478A48894938
:102388001229BAE54625E0F54A754B00854B82F5DA
:1023980083E493B4FF037F0022054BE54B700205ED
:1023A8004A854B82854A83E493F54C740193F54D35
:1023B800E54CB54518E54D6014AB47AA48A949E571
:1023C8004A854BF0120E901229BA7F0122E54CB4CF
:1023D800FF0BE54DB4FF061229BA7F00227B007A75
:0E23E80000794A1225A0EF70B81229BA7F00C2
:0123F60022C4
:082260007B007A007933AD31F7
:082268008B3E8A3F89408D4145
:10227000E4F544F5451229BAE54125E0FEE42401E0
:10228000FFE43EF5428F4385438285428374019388
:10229000F546B43314AB3EAA3FA940E5428543F06E
:1022A000120E901229BA7F0122E546B4770CE5455B
:1022B000454470068542448543457B007A00794257
:1022C0001225A0EF70C1E5454544700CAD41FF12E9
:1022D000295A1229BA7F0022AB3EAA3FA940E54401
:0B22E0008545F0120E901229BA7F0114
:0122EB0022D0
:101CF4007543007544007545377546007547007592
:0C1D040048367B007A007935AF34AE33EE
:0A1D10008E3E8F3F8B408A418942CE
:101D1A008F828E837401937002FF221229BA853F43
:101D2A0082853E83740293F5497F03E53F2403F5D8
:101D3A004CE4353EF54BEFC3940F5016854C828523
:101D4A004B83E493B4FF0B0F054CE54C70E8054B4D
:101D5A0080E4BF0F061229BA7F0022E5414542609E
:101D6A0011853F82853E83E493AB40AA41A9421282
:101D7A000D30E54445456043AB43AA44A945E4F523
:101D8A00F0120E90E4F54AE54AC39549502DAB434B
:101D9A00AA44A945120DF575F000120E90E54C25DE
:101DAA004AF582E4354BF583E493FFAB43AA44A991
:101DBA0045E48FF0120E58054A80CCE54745486045
:101DCA000BAB46AA47A948E549120D301229BA7F3A
:011DDA000107
:011DDB0022E5
:0A24DF008E368F378B388A39893A20
:1024E9008F828E837401937002FF221229BA7F03AF
:1024F900E5372403F53CE43536F53BEFC3940F503B
:1025090016853C82853B83E493B4FF0B0F053CE5BC
:102519003C70E8053B80E4BF0F061229BA7F002210
:10252900E539453A6011853C82853B83E493AB38B4
:0C253900AA39A93A120D301229BA7F010C
:012545002273
:082643008F2A8B2B8A2C892DB4
:10264B007531017B007A00792E853142AF2A122831
:10265B00C47A0009AD2EAF2A12237EEF601F852BA3
:10266B0043852C44852D45754600754700754800FC
:10267B007B007A007900AF30AE2F021D100531E5DB
:08268B0031D3940240BD7F0031
:012693002224
:0826D7008F2E8B2F8A30893110
:1026DF007535017B007A007932853542AF2E12288D
:1026EF00C47A0009AD32AF2E12237EEF600DAB2FEF
:1026FF00AA30A931AF34AE330224DF0535E535D327
:06270F00940240CF7F00A0
:0127150022A1
:101DDC00AD327F7712295A853242AB39AD30AC2FF8
:021DEC00AF2E18
:081DEE008F3E8C3F8D408B41BC
:101DF6007B007A007943AD4212237EEF601BAD442F
:101E0600AC43AF40AE3F122116EF700AAD44AC436F
:101E1600FF12297080037F01227B007A007943AF8D
:101E260042122546EF7015E54225E0F5437544005C
:101E3600FEAF4412285B1229BA7F0022AE43AF449C
:101E4600AD07AC06AF3E122860E54175F002A4D39B
:101E5600940CE5F0648094805013E5442401FFE47B
:101E66003543FEAD07FC7F77122860800BE54424DE
:101E760001FFE4354312285AE5442402FFE43543C2
:101E8600FEAD07FCAF411228607901E9D3954150B8
:101E960024AF40E540E544240FFDE43543FCE9FB6F
:101EA600C3ED9BFDEC9400FC122860E53FF5407500
:0A1EB6003F000980D61229BA7F010F
:011EC00022FF
:08210E00AD34AC33AF30AE2F4D
:082116008E458F468C478D4871
:10211E0085474A85484B854B82854A83740193B423
:10212E0033037F00221229BA7402254BF54BE43596
:10213E004AF54A854B82F583E493F549054BE54B09
:10214E007002054AE4FD854B82854A83E493B4FF11
:10215E0011EDD3940C500B054BE54B7002054A0D57
:10216E0080E4E54975F002A4FFC3ED9FE5F06480BD
:10217E00F8748098500BE5482401FFE43547122887
:10218E005A7901E9D39549501DAF46E546E9FDC39D
:10219E00E54B9DFDE54A9400FC122860E545F546A9
:0B21AE007545000980DD1229BA7F0191
:0121B9002203
:0606FB008F2E8C2F8D30C4
:10070100E4F53CF53DD3E53094FFE52F9400400539
:1007110075390280037539017D017B007A007931D9
:100721008D42AF2E1228C4E53125E0F53375340032
:10073100853482F583E4937005AF311228D2853474
:1007410082853383E493FFB4FF0874392DF8E4F60E
:10075100801274392DF8A605EFB477028D3DEFB400
:1007610033028D3C0DBD03B21229BAE53A701EE584
:100771003B701AFB7A007931754201AF2E1228C401
:10078100AD317F7712295A853142021DE6E53A6083
:1007910007E53B60030208B3E53D7007E53C7003E4
:1007A1000208B3E53D70030208397B007A00793114
:1007B100F542AF2E1228C4122376EF604612210EA5
:1007C100EF600302098FAD34AC33FF12297085311C
:1007D10042121DE6EF600302098F1228B6121DDCDA
:1007E100122260EF700302098F121CF4EF700302F2
:1007F100098F853242AB36AD38AC37AF35121DEEBD
:1008010002296A853142121DE6EF600302098F1247
:1008110028B6121DDC122260EF700302098F121C30
:10082100F4EF700302098F853242AB36AD38AC3735
:10083100AF35121DEE02296A7B007A007931853CC1
:1008410042AF2E1228C4122376EF603412210EEF2C
:10085100600302098FAF3C1228B8121DDC1222601E
:10086100EF700302098F121CF4EF700302098F85E8
:100871003242AB36AD38AC37AF35121DEE02296AC4
:10088100AF3C1229398F427B001228BE121DDC12A7
:100891002260EF700302098F121CF4EF700302094A
:1008A1008F853242AB36AD38AC37AF35121DEE0213
:1008B100296A7B007A007932853D42AF2E1228C425
:1008C1007A0019853C42AF2E1228C4122376EF60BC
:1008D1006712210EEF600302098FFB7A007933ADB5
:1008E10032AF2E12237EEF602F12210EEF60030232
:1008F100098F121DE3122260EF700302098F121C8F
:10090100F4EF700302098F853242AB36AD38AC3754
:10091100AF35121DEE02296A121DE3122260EF604B
:100921006D121CF4EF6067853242AB36AD38AC37DF
:10093100AF35121DEE02296A7B007A007933AD32A0
:10094100AF2E12237EEF602612210EEF7040121D92
:10095100E3122260EF6037121CF4EF6031853242FE
:10096100AB36AD38AC37AF35121DEE02296A121D18
:10097100E3122260EF6017121CF4EF60118532421E
:0E098100AB36AD38AC37AF35121DEE12296A19
:01098F002245
:101FD20060600042000000000000000000000000FD
:101FE20000000000000000000000000000000000EF
:101FF20000000000000000000000000000000000DF
:1020020000000000000000000000000000000000CE
:1020120000000000000000000000000000000000BE
:1020220000000000000000000000000000000000AE
:10203200000000004800000000000000000000480E
:10204200003AFFFFFFFFFFFFFFFF4800A2FFFFFF75
:05205200FFFFFFFFFF8E
:04136C008F238D241A
:10137000EAF52AEBF52BE527F52CE528F52DE4F524
:101380002F7456252FF8E4F6052FE52FB432F2D24C
:10139000059000F3E0FFC4540F25E024D0F582E46B
:1013A0003400F583EF540FFFE0FEA3E0A8070880A8
:1013B00005CEC313CE13D8F930E004D20D8002C29B
:1013C0000D9000EEE0A320E706200D030215501259
:1013D00029951229AAD2059000F3E0900008F0F5B3
:1013E00029852999C215AF291228A09000097406F1
:1013F000F0F5293015FD852999C215AF291228A0CD
:1014000090000AE52AF0F5293015FD852999C215C5
:10141000AF291228A090000BE52BF0F5293015FD1F
:10142000852999C215AF291228A090000CE52CF04F
:10143000F5293015FD852999C215AF291228A090EC
:10144000000DE52DF0F5293015FD852999C215AF60
:10145000291228A03015FD7851E690000EF0F529EC
:10146000F599C2153015FD7853E690000FF0F52977
:10147000F599C2153015FD1229A01229BA752E88CA
:10148000C216C20C20160FE52E600B152E7F647E4F
:101490000012297E80EEE52E7004D20C8019900097
:1014A0000EE0FF785CE6B5070CA3E0FF08E6B507A1
:1014B00004C20C8002D20C300C487530007531012A
:1014C0009000F3E0FD540FFFE531AE30A80708802F
:1014D00005C333CE33CED8F9F5318E30EDC4540F79
:1014E00025E024D0F582E43400F583C083C082E097
:1014F0004530FFA3E04531D082D083CFF0A3EFF099
:10150000804E7530FF7531FEE4F52F9000F3E0FD5D
:10151000540FFFE52FC39F5013E53125E0FFE53061
:1015200033F530EF4401F531052F80DFEDC4540F62
:1015300025E024D0F582E43400F583C083C082E046
:101540005530FFA3E05531D082D083CFF0A3EFF028
:101550009000F3E0C39524400CE523F09000EEE00A
:0D156000547FF080069000F3E004F0C20517
:01156D00225B
:03000000020200F9
:0C020000787FE4F6D8FD75819C0202476F
:100C2100E709F608DFFA8046E709F208DFFA803EB5
:100C310088828C83E709F0A3DFFA8032E309F608A2
:100C4100DFFA8078E309F208DFFA807088828C830A
:100C5100E309F0A3DFFA806489828A83E0A3F608BE
:100C6100DFFA805889828A83E0A3F208DFFA804C98
:100C710080D280FA80C680D4806980F2803380106F
:100C810080A680EA809A80A880DA80E280CA8033D8
:100C910089828A83ECFAE493A3C8C582C8CCC58350
:100CA100CCF0A3C8C582C8CCC583CCDFE9DEE78020
:100CB1000D89828A83E493A3F608DFF9ECFAA9F09F
:100CC100EDFB2289828A83ECFAE0A3C8C582C8CCF5
:100CD100C583CCF0A3C8C582C8CCC583CCDFEADE0E
:100CE100E880DB89828A83E493A3F208DFF980CC70
:100CF10088F0EF60010E4E60C388F0ED2402B40469
:100D01000050B9F582EB2402B4040050AF2323450F
:060D11008223900C7173B7
:100D1700BB010689828A83E0225002E722BBFE02DA
:090D2700E32289828A83E493220D
:100D3000BB010689828A83F0225002F722BBFE01A2
:020D4000F3229C
:100D4200EF8DF0A4A8F0CF8CF0A428CE8DF0A42EC5
:020D5200FE227F
:100D5400BC000BBE0029EF8DF084FFADF022E4CC83
:100D6400F875F008EF2FFFEE33FEEC33FCEE9DEC4C
:100D7400984005FCEE9DFE0FD5F0E9E4CEFD22ED92
:100D8400F8F5F0EE8420D21CFEADF075F008EF2FDC
:100D9400FFED33FD4007985006D5F0F222C398FDCD
:050DA4000FD5F0EA226A
:100DA900C2D5EC30E709B2D5E4C39DFDE49CFCEE65
:100DB90030E715B2D5E4C39FFFE49EFE120D54C37C
:100DC900E49DFDE49CFC8003120D5430D507C3E477
:060DD9009FFFE49EFE22D4
:100DDF00C5F0F8A3E028F0C5F0F8E582158270029F
:060DEF001583E038F0223C
:100DF500BB010A89828A83E0F5F0A3E022500687C9
:100E0500F009E71922BBFE07E3F5F009E31922898A
:0B0E1500828A83E493F5F074019322BD
:100E2000BB0110E58229F582E5833AF583E0F5F010
:100E3000A3E0225009E92582F886F008E622BBFEED
:100E40000AE92582F8E2F5F008E222E5832AF58333
:080E5000E993F5F0A3E99322F8
:100E5800BB010789828A83020DDF500B09C5F02781
:100E6800F7C5F01937F722BBFE0D09F8E325F0F3B3
:100E7800C5F019E338F322F889828A83740193252F
:080E8800F0C5F0F8E4933822F4
:100E9000BB010A89828A83F0E5F0A3F0225006F7AD
:0F0EA00009A7F01922BBFE06F3E5F009F31922AA
:10292700C3EE6480948040028007C3E49FFFE49E67
:02293700FE227E
:10020C0002191CE493A3F8E493A34003F68001F2D3
:10021C0008DFF48029E493A3F85407240CC8C333F3
:10022C00C4540F4420C8834004F456800146F6DFC2
:10023C00E4800B0102040810204080901F96E47E9D
:10024C00019360BCA3FF543F30E509541FFEE493B7
:10025C00A360010ECF54C025E060A840B8E493A37E
:10026C00FAE493A3F8E493A3C8C582C8CAC583CAA9
:10027C00F0A3C8C582C8CAC583CADFE9DEE780BE61
:012057000088
:00000001FF
